:020000040000FA
:040000006E303A28FC
:08000800A000030EA100831209
:1000100005191028831601178312B23081002B288E
:1000200083160113831203140B190310A80DA90DD5
:10003000AA0DAB0DAC0DAC16FF302C02031D2B2806
:10004000FA302B02031D2B2831152A08AF0029088E
:10005000AE002808AD008B100B11210E8300A00EFE
:04006000200E090065
:0C007400203084008001840A6030040207
:10008000031C3C281230B00084218316FF2390000B
:10009000831283160C308505870183128501870141
:1000A000073099000030831691008312C830831600
:1000B0008100831231309000003083168C0083124F
:1000C00010308B00831600309B001C141A0883121A
:1000D000BC00831610309B001C141A088312BD004C
:1000E0009D2181018E018F010B118B100B108C0152
:1000F0008B17892031198C206821B30B87280310B6
:1001000085190314B90DF0303902031911219E210C
:10011000792864003210080031110130B7008B13C8
:100120002030370783169B001C141A088312A40082
:100130001030370783169B001C141A088312A30083
:10014000A6000230A6060030370783169B001C1459
:100150001A088312A200A7000130A7068B17321CD1
:10016000B72822090339A200A309A409A509240874
:100170002F02031D0B2923082E02031D0B29220821
:100180002D02031D0B2901303702031DCC283D1819
:10019000CC283D143E14852102303702031DD5289A
:1001A000BD18D528BD143E14882103303702031D25
:1001B000DE283D19DE283D153E148B210430370220
:1001C000031DE728BD19E728BD153E148E21053013
:1001D0003702031DF0283D1AF0283D163E149121E8
:1001E00006303702031DF928BD1AF928BD163E1442
:1001F000942107303702031D02293D1B02293D17B8
:100200003E14972108303702031D0B29BD1B0B2913
:10021000BD173E149A21B70A0930370203180800A7
:100220008F280130B600B300B400B500B7008501D7
:100230008701B1138920B30B3729031085190314E3
:10024000B90DF030390203195E29B41F8501B41FBE
:100250008701B40B37293708B6080319B60003190C
:100260003529FF3085008700B6039630B400311D74
:100270001A293111321C41292D090339AD00AE096B
:10028000AF092F1C1A298E018F010C1C1A290C1082
:100290002E1E1A298B1320303707BB002F08BA00F7
:1002A000712110303707BB002E08BA0071210030D1
:1002B0003707BB002D08BA0071218B178501870114
:1002C000B70AB60109303702031C1A299D2108001C
:1002D0003E1C08003E101030BB003D08BA007121E2
:1002E00008008B133A0883161C159A003B089B00E4
:1002F00055309D00AA309D009C1464009C187D29F7
:100300001C1183128B17080008000130BD00080083
:100310000230BD0008000430BD0008000830BD00F8
:1003200008001030BD0008002030BD00080040303B
:10033000BD0008008030BD00080008008F080319C8
:1003400008008F0107303D050319962A02303D054C
:10035000031D51105408EB3C031805125118B32922
:10036000D40BBE29B829D4035408C83C031CBE29A9
:100370000516F530D4005108013AD10002303D0590
:10038000031DD1105508E63C03188512D118CB295E
:10039000D50BD629D029D5035508B93C031CD6293D
:1003A0008516F030D5005108023AD10002303D05E3
:1003B000031D51115608DC3C031805105119E3299F
:1003C000D60BEE29E829D6035608B63C031CEE29C5
:1003D0000514E630D6005108043AD10002303D053C
:1003E000031DD1115708F03C03188510D119FB29C2
:1003F000D70B062A002AD7035708D73C031C062A26
:100400008514FA30D7005108083AD10002303D0572
:10041000031D51125808E03C03188710511A132A83
:10042000D80B1E2A182AD8035808C13C031C1E2AC0
:100430008714EA30D8005108103AD10006303D0543
:10044000031DD1125908D43C03180711D11A2B2AC5
:10045000D90B362A302AD9035908A73C031C362A5F
:100460000715DE30D9005108203AD10006303D058D
:10047000031D51135A08BF3C03180710511B432A90
:10048000DA0B4E2A482ADA035A089C3C031C4E2AEF
:100490000714C930DA005108403AD10006303D0552
:1004A000031DD1135B08D73C03188712D11B5B2AAD
:1004B000DB0B662A602ADB035B08BE3C031C662A52
:1004C0008716E130DB005108803AD10006303D0547
:1004D000031D52105C08F13C031807125218732ACE
:1004E000DC0B7E2A782ADC035C08CF3C031C7E2AC6
:1004F0000716FB30DC005208013AD20006303D05F9
:10050000031DD2105D08E93C03188711D2188B2A0D
:10051000DD0B962A902ADD035D08B23C031C962A67
:100520008715F330DD005208023AD20018303D053D
:100530000319E62ABD1DA22A54083C3C031CA22A2A
:1005400085018701D40B0800D0034630D4000B305E
:100550005002031DAC2A05160A305002031DB12AB1
:10056000851609305002031DB62A051408305002C2
:10057000031DBB2A851407305002031DC02A8714AF
:1005800006305002031DC52A071505305002031D11
:10059000CA2A071404305002031DCF2A87160330DD
:1005A0005002031DD42A071602305002031DD92A17
:1005B000871501305002031DDD2A12305002031C42
:1005C0000800850187010C30D000080020303D056F
:1005D0000319302BD40BF12A0508103A850082301C
:1005E000D400D50BF82A0508203A85007D30D500C7
:1005F000D60BFF2A0508013A85007330D600D70BC9
:10060000062B0508023A85008730D700D80B0D2B42
:100610000708023A87007730D800D90B142B070857
:10062000043A87006B30D900DA0B1B2B0708013A1C
:1006300087005630DA00DB0B222B0708203A8700B0
:100640006E30DB00DC0B292B0708103A870088305E
:10065000DC00DD0B302B0708083A87008030DD0016
:1006600040303D050319A72B5408E63C031805123A
:10067000D40B562B0516F030D4002130DE070318BA
:10068000542BB130D507FA30D607C830D7076430BD
:10069000D8079630D907BE30DA07AA30DB079A3080
:1006A000DC07C430DD07562B8030BD005508823C86
:1006B00003188512D50B5F2B85168C30D500560894
:1006C000653C03180510D60B682B05146F30D60057
:1006D0005708913C03188510D70B712B85149B305C
:1006E000D7005808D73C03188710D80B7A2B8714EB
:1006F000E130D8005908503C03180711D90B832B5F
:1007000007155A30D9005A08873C03180710DA0B2E
:100710008C2B07149130DA005B08BD3C031887125C
:10072000DB0B952B8716C730DB005C08703C031889
:100730000712DC0B9E2B07167A30DC005D08A73C05
:1007400003188711DD0BA72B8715B130DD00803032
:0E0750003D050319AE2B85018701DE0108006F
:084000000B00030002000600A2
:02400E00CC01E3
:10420000010078007A007C007E007B0079007F004E
:104210007D007A0078007E007C00FF00FF00FF0038
:104220000000F200F600FA00FE00F200F600FA00CC
:10423000FE00F200F600FA00FE00FF00FF00FF00A3
:10424000010005000500050005000900090009003E
:1042500009000D000D000D000D00FF00FF00FF0024
:10426000FF00FF00FF00FF00FF00FF00FF00FF0056
:10427000FF00FF00FF00FF00FF00FF00FF00FF0046
:10428000FF00FF00FF00FF00FF00FF00FF00FF0036
:10429000FF00FF00FF00FF00FF00FF00FF00FF0026
:1042A000FF00FF00FF00FF00FF00FF00FF00FF0016
:1042B000FF00FF00FF00FF00FF00FF00FF00FF0006
:1042C000FF00FF00FF00FF00FF00FF00FF00FF00F6
:1042D000FF00FF00FF00FF00FF00FF00FF00FF00E6
:1042E000FF00FF00FF00FF00FF00FF00FF00FF00D6
:1042F000FF00FF00FF00FF00FF00FF00FF00DD00E8
:00000001FF
